:020000040800F2
:1000000060110020C9010008CD170008D9110008AF
:10001000C9170008050500083B2F00080000000074
:10002000000000000000000000000000CD1D0008DE
:10003000350E000800000000051A0008CD26000853
:10004000E3010008E3010008E3010008E301000800
:10005000E3010008E3010008E3010008E3010008F0
:10006000E3010008E3010008E3010008E3010008E0
:10007000E3010008E3010008E3010008E3010008D0
:10008000E3010008E3010008E3010008E3010008C0
:10009000892E0008E3010008E3010008E3010008DD
:1000A000E3010008E3010008E3010008E3010008A0
:1000B000A1270008E3010008E3010008E3010008AC
:1000C000E3010008E3010008E3010008E301000880
:1000D000E3010008E301000855290008E3010008D6
:1000E000E3010008E30100081F2C000800F002F8FB
:1000F00000F05AF80AA090E8000C82448344AAF168
:100100000107DA4501D100F04FF8AFF2090EBAE865
:100110000F0013F0010F18BFFB1A43F0010318473B
:10012000E8380000083900000A444FF0000C10F8CD
:10013000013B13F0070408BF10F8014B1D1108BF65
:1001400010F8015B641E05D010F8016B641E01F805
:10015000016BF9D113F0080F1EBF10F8014BAD1C55
:100160000C1B09D16D1E58BF01F801CBFAD505E073
:1001700014F8016B01F8016B6D1EF9D59142D6D3CD
:10018000704700000023002400250026103A28BFF5
:1001900078C1FBD8520728BF30C148BF0B607047F9
:1001A0001FB51FBD10B510BD00F099F81146FFF73F
:1001B000F7FF02F0F3FE00F0B7F803B4FFF7F2FF29
:1001C00003BC00F0BFF80000094880470948004719
:1001D000FEE7FEE7FEE7FEE7FEE7FEE7FEE7FEE7F7
:1001E000FEE7FEE704480549054A064B7047000054
:1001F00041270008ED000008600B0020601100207E
:10020000600D0020600D00204FF0000200B5134685
:1002100094469646203922BFA0E80C50A0E80C5026
:10022000B1F12001BFF4F7AF090728BFA0E80C50D7
:1002300048BF0CC05DF804EB890028BF40F8042BD0
:1002400008BF704748BF20F8022B11F0804F18BF3D
:1002500000F8012B704700004FF0013C50F8042BD0
:1002600051F8043B9A4221D1A2EB0C03934313EAC9
:10027000CC1317D150F8042B51F8043B9A4215D1F6
:10028000A2EB0C03934313EACC130BD150F8042BCD
:1002900051F8043B9A4209D1A2EB0C03934313EAB1
:1002A000CC13DBD04FF00000704700BFD01A01BA6A
:1002B000B1FA81F101F0180122FA01F0CB40C1F14D
:1002C0002001DBB2C0B2C01A2CFA01F3D11A91435B
:1002D00011EAC311E6D17047704770477047754601
:1002E00000F02CF8AE4605006946534620F00700A2
:1002F000854618B020B5FFF775FFBDE820404FF0E8
:1003000000064FF000074FF000084FF0000B21F0FF
:100310000701AC46ACE8C009ACE8C009ACE8C009CC
:10032000ACE8C0098D46704710B50446AFF30080B5
:100330002046BDE81040FFF740BF0000004870476E
:10034000FC0A002001491820ABBEFEE7260002008F
:100350007047000008B58020ADF8000003208DF83C
:10036000020010208DF803006946044800F019FED1
:100370008021024800F0F1FE08BD000000080140A5
:1003800010B500F015F800F097F8FFF7E3FF10BD87
:1003900010B50121044800F0E0FE00200349087078
:1003A000142000F055FD10BD000C0140B1000020EC
:1003B00000B587B00121480401F07AFB2B4802F018
:1003C0000FFB0420ADF8180003208DF81A00182048
:1003D0008DF81B0006A9264800F0E3FD0820ADF8C3
:1003E000180004208DF81B0006A9214800F0D9FD53
:1003F0004FF4165002900020ADF80C00ADF80E003E
:10040000ADF81000ADF814000C20ADF8120002A9F0
:10041000164802F08FFB4FF4A06001F011FA26207D
:100420008DF8040001208DF805008DF806008DF888
:10043000070001A801F0CCF940F226610B4802F058
:10044000B4FA40F22771094802F0AFFA012240F2F3
:100450002551064802F049FB4021044802F09CFA6D
:100460000121024802F0B0FA07B000BD004400408C
:100470000008014010B504462146074802F0CBFBB6
:1004800000BF4021044802F0F9FA0028F9D04021C9
:10049000014802F081FA10BD0044004070B50546E5
:1004A0000E46002404E0285DFFF7E4FF601CC4B2A0
:1004B000B442F8DB70BD000008B50120ADF80000C3
:1004C00003208DF8020010208DF8030069460448CF
:1004D00000F067FD0121024800F041FE08BD000068
:1004E000000C014010B50121044800F038FE012045
:1004F00003490870142000F0ABFC10BD000C014053
:10050000B100002000BFFEE70146CAB20B1243EA69
:100510000220704708B50020009022E1974800882B
:1005200000F00F00964908700846007800287CD13A
:1005300094480068944908800846008800F030001C
:10054000924908809048008800F440508E49088005
:100550008C4909684BF6BF7201EA020080F4005032
:1005600080F0200040F4004141F08001854A116094
:100570008248008800F0100090BB1046006848F6E2
:100580000F7108401146086000F028FE7D49096897
:100590004BF6BF7201EA02007B49098801F48051E1
:1005A00009B180F480507849098801F4005109B1FB
:1005B00080F400507549098801F0100109B180F0FC
:1005C00010007249098801F0200109B180F0200073
:1005D00081B241F4004141F080016A4A116008BDD6
:1005E000FFE76848006880B20090BDF8000000F4A2
:1005F0000060B0B363480068C0F30E0048F68F7126
:1006000008406049086001F06DFD5E4909684BF6DD
:10061000BF7201EA02005C49098801F4805109B106
:1006200080F480505849098800E056E001F40051F8
:1006300009B180F400505549098801F0100109B151
:1006400080F010005149098801F0200109B180F0C3
:10065000200081B241F4004141F08001494A11601B
:10066000BDE7FFE7BDF8000000F40040002878D0A7
:1006700044480068C0F30E0048F68F7108404149B5
:10068000086001F083F93F4909684BF6BF7201EA3F
:1006900002003D49098801F4805109B180F480507D
:1006A0003949098801F4005109B180F400503749F3
:1006B000098801F0100109B180F010003349098860
:1006C00001F0200109B180F0200081B241F4004125
:1006D00041F080012B4A116081E7294800782C49BC
:1006E00001EB8000D0F8000C80B20090BDF8000053
:1006F00000F40040C0B12248007801EB8000D0F83F
:10070000000CC0F30E0048F68F7108401C490978B0
:100710001F4A02EB8101C1F8000C19490978491EF2
:100720001C4A52F821008047BDF8000000F080000C
:10073000B8B113480078164901EB8000D0F8000CDE
:1007400048F60F7108400E490978114A02EB810101
:10075000C1F8000C0A490978491E0F4A52F82100D5
:10076000804708484430006880B20449088000F49B
:10077000004000287FF4D2AE00BF30E7F000002038
:10078000BC000020005C0040D0000020D20000200F
:100790000050004018010020FC0000200B4A02EB32
:1007A0008001D1F8001C01F4804171B102EB80019D
:1007B000D1F8001C48F68F7211404CF280021143B0
:1007C000024B03EB8002C2F8001C7047005000404F
:1007D0000B4A02EB8001D1F8001C01F0400171B11D
:1007E00002EB8001D1F8001C48F68F72114048F2EC
:1007F000C0021143024B03EB8002C2F8001C704799
:1008000000500040084A02EB8001D1F8001C48F675
:100810008F62114048F280021143034B03EB8002C8
:10082000C2F8001C704700000050004000F08051EA
:1008300011B10349086001E00249486070470000B7
:10084000040402400000024021B1026842F00102AB
:10085000026004E002684FF6FE731A4002607047BF
:1008600001684FF6FE721140016000210160416095
:100870008160C1604B49884208D14A4908394968BA
:1008800041F00F01474A083A51608AE04549143166
:10089000884208D143490839496841F0F001414A8A
:1008A000083A51607DE03F492831884208D13D49EE
:1008B0000839496841F470613A4A083A516070E079
:1008C00038493C31884208D136490839496841F4F1
:1008D0007041344A083A516063E0324950318842ED
:1008E00008D130490839496841F470212D4A083A45
:1008F000516056E02B496431884208D129490839B2
:10090000496841F47001274A083A516049E0254995
:100910007831884208D123490839496841F070612B
:10092000204A083A51603CE01F49884206D1011F25
:10093000096841F00F01021F116032E01A491431B9
:10094000884208D11849091F096841F0F001164A88
:10095000121F116025E014492831884208D112493C
:10096000091F096841F470610F4A121F116018E0F5
:100970000D493C31884208D10B49091F096841F4EF
:100980007041094A121F11600BE00749503188423B
:1009900007D10549091F096841F47021024A121F55
:1009A0001160704708000240080402400146486890
:1009B00080B2704701460020002201F0805313B13D
:1009C000054B1A6801E0054B1A6802EA01030BB1F6
:1009D000012000E0002070470004024000000240B7
:1009E00010B50022026847F6F0739A430C6A8B68D0
:1009F00023430C6923434C6923438C692343CC690B
:100A000023434C6A23438C6A23431A430260CB6816
:100A100043600B6883604B68C36010BD41607047E2
:100A20002DE9F0472848006800F110052E88264877
:100A30000068077AD6B9042F18D124480078012815
:100A40000FD100212248006880B2801C214A42F860
:100A5000101030202049088000BF00201B4908707A
:100A600003E0072710201C49088027E0AC88A64235
:100A700001D8042000E002200746B44200D93446E1
:100A8000A0B2A96888478046002000F07BFB814621
:100A9000A2B24946404602F053FAA1B2002001F04A
:100AA00049FA2888001B2880688820446880302004
:100AB0000949088000020949088000BF0249096805
:100AC0000F72BDE8F0870000C0000020B8000020D1
:100AD000505C004000600040D2000020D0000020A8
:100AE0002DE9F0412848006800F110042688A0682C
:100AF000C0B1BEB1A588B54200D93546A8B2A1683B
:100B0000884707462088401B2080608828446080F2
:100B1000002000F027FB8046AAB24146384600F08C
:100B20005DFF00BF208850B14FF440501749088046
:100B30000021084601F0FEF9302015490880208880
:100B4000A188884204DB03200F490968087218E075
:100B50002088002804DD05200B490968087210E090
:100B6000208870B9062008490968087200210948E0
:100B7000006880B2801C084A42F8101030200449F6
:100B80000880BDE8F0810000C0000020D0000020F7
:100B9000D2000020505C0040006000402DE9F84F7A
:100BA0009B48006845780027BA46062D1BD1984817
:100BB0000068007800F07F00002813D1944909688C
:100BC0008878012803D193490968CF690AE002288F
:100BD00003D1904909680F6A04E0032802D18D49C6
:100BE00009684F6A94E0002D64D189480068408804
:100BF00000285FD186480068C08802285AD18448FE
:100C000000680079002855D181480068007800F01C
:100C10007F0028B97E480068808808B97E4F77E059
:100C20007B480068007800F07F00012810D17849E7
:100C300009684879774909688A690021904700283E
:100C400066D173480068807A002861D0724F5FE0F7
:100C50006F480068007800F07F00022858D16C4887
:100C60000068407900F00F0669480068407900F09C
:100C7000700967480068407900F0800038B1674922
:100C800001EB8600D0F8000C00F0300806E0634964
:100C900001EB8600D0F8000C00F440586048007862
:100CA000B04235D9B9F1000F32D1B8F1000F2FD0D1
:100CB000594F2DE0082D07D155480068007800F005
:100CC0007F0028BB574F23E00A2D21D150480068F0
:100CD000007800F07F0001281AD14D480068807A22
:100CE000B0B14B480068408890B949480068007925
:100CF00070B947480068C088012809D1444909688B
:100D00004879444909688A690021904700B9464FEB
:100D100057B13F480068A0F812A03D4800688761BD
:100D20000020B84700240FE0394A12685078394A49
:100D30001268116988470446032C05D109203449FB
:100D400009680872BDE8F88F31480068008A4FF6DC
:100D5000FF71884204D109202D4909680872F1E722
:100D6000022C03D02A480068008A20B908202849AC
:100D700009680872E6E726480068007800F08000FD
:100D8000E0B323480068C088009021480068008ACA
:100D90000099884204D91E4900980968088223E016
:100DA0001B480068008A1A490968C98888421BDA0A
:100DB00017480068008A1749096891F82C10884282
:100DC00003DA0020194908700EE011480068008A13
:100DD0001049096891F82C1090FBF1F201FB120008
:100DE00010B90120114908700A48006890F82C10C9
:100DF000074800688182FFF713FE07E0FFE7032042
:100E000003490968087200030949088000BF99E78F
:100E1000C0000020C40000208523000800500040CE
:100E2000380100200923000859230008B8000020D9
:100E3000D0000020704710B50246002404E04FF4B3
:100E40007A7000F005F8521E9442F8D310BD0000ED
:100E500001B504490098086000BF024800680028F6
:100E6000FBD108BD34000020012001490870704703
:100E7000D4000020014908607047000014040140BC
:100E8000002123498279002A3AD00A461268036871
:100E90009A430B461A600A1D126803689A430B1D99
:100EA0001A60027911440A6803681A430A60184AF2
:100EB0000832126803689A43154B08331A601A1DEA
:100EC000126803689A43124B0C331A604279102A55
:100ED0000ED11A1F126803681A430D4B08331A60AB
:100EE0001A1D126803681A43094B0C331A600DE08F
:100EF0000749427911440A6803681A430A6005E009
:100F0000027911440A6803689A430A607047000036
:100F1000000401400320014908607047D00100200F
:100F200010B500F029F800F001F810BD0EB5012150
:100F3000084600F0BDFD40F2E730ADF80400472060
:100F4000ADF800000020ADF80600ADF802008DF805
:100F5000080069464FF0804001F09EFC012188079F
:100F600001F06EFC01221146900701F08CFC01217A
:100F7000880701F06BFC0EBD08B54FF4E06000F08F
:100F80005FFC1C208DF8000000208DF8010003207C
:100F90008DF8020001208DF80300684600F018FC6F
:100FA00008BD2DE9F041024600250026002000235F
:100FB0000024002791F803C00CF00F0591F803C03E
:100FC0000CF0100CBCF1000F03D091F802C04CEAF9
:100FD000050591F800C0BCF1000F31D01468002065
:100FE0002BE04FF0010C0CFA00F3B1F800C00CEA52
:100FF00003069E4220D183004FF00F0C0CFA03F73A
:10100000BC4305FA03FC4CEA040491F803C0BCF1AC
:10101000280F06D14FF0010C0CFA00FCC2F814C0E6
:101020000AE091F803C0BCF1480F05D14FF0010C64
:101030000CFA00FCC2F810C0401C0828D1D3146080
:10104000B1F800C0BCF1FF0F34DD546800202EE081
:1010500000F1080C4FF0010808FA0CF3B1F800C0D9
:101060000CEA03069E4221D183004FF00F0C0CFACC
:1010700003F7BC4305FA03FC4CEA040491F803C0EF
:10108000BCF1280F05D100F1080C08FA0CF8C2F8E1
:10109000148091F803C0BCF1480F07D100F1080C8F
:1010A0004FF0010808FA0CF8C2F81080401C08281C
:1010B000CED35460BDE8F081F0B50A460023002489
:1010C0000021002500F00046B6F1004F02D11D4E70
:1010D000F16901E01B4E7168C0F3034583B200F46F
:1010E0004016B6F5401F08D121F07061154E7668A4
:1010F00026F07066134F7E6012E000F48016B6F59D
:10110000801F06D1032606FA05F4A14341F0706161
:1011100006E0460D360103FA06F6B14341F0706170
:1011200022B1460D360103FA06F6314300F00046BF
:10113000B6F1004F02D1034EF16101E0014E716042
:10114000F0BD0000000001400246002093680B4003
:101150000BB1012000E00020704741617047016140
:101160007047000001460548006880B200EBC100EE
:10117000001D034A32F8100080B27047505C0040F6
:101180000060004001460548006880B200EBC100E5
:10119000034A32F8100080B270470000505C0040F3
:1011A0000060004070B50A480468001D0568001D15
:1011B0000668344454B108220649204600F046F837
:1011C000042204491031284600F040F870BD0000A8
:1011D000E8F7FF1FD700002000BFFEE710B5184852
:1011E0000068047A022C01D0042C05D1FFF718FC0A
:1011F00013480068047A1CE0062C19D110480068D6
:10120000407805280ED10E480068007800F07F0075
:1012100040B90B490968C87800F0E2FD094909683E
:10122000086A80470849096888688047082400E000
:101230000824034909680C7200F0E6FB10BD0000A9
:10124000C0000020CC000020C400002030B50B46B8
:10125000002100BF16E00A24B4EB107F05D930242A
:1012600004EB107403F8114005E0412404EB107402
:101270000A3C03F81140000100254C00641C1D5578
:101280004C1CE1B29142E6DB30BD000070B5044673
:101290000025062C18D118480068007800F07F005F
:1012A000012811D114480068407968B912480068D3
:1012B0008078222801D1114D10E00F480068807815
:1012C00021280BD10E4D09E00B480068007800F092
:1012D0007F00212802D1032C00D10A4D0DB9022034
:1012E00070BD05480068856100210348006841829F
:1012F0000020A8470020F3E7C00000206113000889
:10130000311300084513000810B504460249204671
:1013100001F010F810BD00009801002010B504463F
:101320000249204601F006F810BD0000900100209F
:1013300010B504460249204600F0FCFF10BD000035
:10134000A8010020014629B90120034A1268108231
:10135000002070470148FCE7C00000203401002055
:1013600010B504460249204600F0E4FF10BD00001D
:10137000A001002070B5054606480068C478042C1A
:1013800001DD002070BD044800EBC401284600F0D8
:10139000D1FFF7E7C0000020B0010020024600297D
:1013A00001DD02207047002A01DD0220FAE700205B
:1013B000F8E7000000B5024606480068007800F033
:1013C0007F00212804D10B2A02D100F069F800BD6A
:1013D0000220FCE7C000002010B500202349096866
:1013E000887222490968C8722148C0791F49096872
:1013F0004872002000F0ECFC4FF40071002000F077
:10140000E1FD1021002000F0A3FD1821002000F0D4
:101410000FFD5821002000F07DFD0020FFF7F2F9BC
:10142000144890F82C10002000F014FD002000F06B
:1014300057FD4FF4C061012000F0C4FD4FF48071EE
:10144000012000F067FD0421012000F073FD002160
:10145000012000F025FD2021012000F079FD002071
:1014600000F0BEFC01200449086010BDC00000204F
:10147000DA3800083C010020D00100200348817ABE
:1014800011B10521024A116070470000C00A002016
:10149000D00100200420014908607047D0010020DD
:1014A00003480068C17803480160002070470000CD
:1014B000C0000020340100207047704710B5FFF7CE
:1014C00071FE002005490968887200F0C1FA01F038
:1014D0000BFD00200249086010BD0000C000002084
:1014E000D001002010B5044608222146812001F0D9
:1014F0000DFD012000F04CFD10BD000010B592B0B4
:1015000000240121084600F0C3FA0121880300F0FD
:10151000CFFA3748FFF7A4F900200490354801902E
:10152000354802901020039000200A9005908020FA
:10153000069040000790800008900020099001A9C3
:101540002B48FFF74DFA0121082000F0D1FA4FF4A3
:101550000040ADF8440018208DF8470003208DF8B6
:10156000460011A92548FFF71CFD22480C3800F061
:10157000E3FB4FF44040ADF830004FF48270ADF81B
:1015800032004FF40060ADF834000020ADF83600B2
:10159000ADF838004FF40070ADF83A000820ADF80F
:1015A0003C000020ADF83E000720ADF840000CA93B
:1015B00010480C3800F0ECFB012202210D480C38D9
:1015C00000F0B0FB01210B480C3800F09FFB00BF7E
:1015D00005E00020084921F81400601C84B2B4F52D
:1015E000806FF6DB00200649088012B010BD0000B5
:1015F000580002400C380040C0020020000C01409E
:10160000B40000202DE9F04105460E464FF4E047B6
:101610004FF4FE48002480240AE005EA040109B1E1
:10162000414600E0394688B2314600F0A1F8641026
:10163000012CF2DABDE8F0812DE9F04104460D46B7
:10164000C4F30726C4F3074704F0FF0829463846C9
:10165000FFF7D8FF29463046FFF7D4FF294640461A
:10166000FFF7D0FFBDE8F0812DE9F04107460D46B8
:1016700016460024022E38D13B48FFF797F9002880
:1016800070D100BF06E057F824003146FFF7D4FFC1
:10169000601CC4B2AC42F6D3002405E03146002001
:1016A00000F066F8601CC4B2142CF7DB00202F4950
:1016B000088005EB4500C000143081B22A48FFF7CE
:1016C000ADF901212848FFF7BFF800BF4FF4003003
:1016D000FFF770F90028F9D000212348FFF7B4F88C
:1016E0004FF40030FFF7A2F83CE0012E3AD11E483B
:1016F0002838FFF75BF9A8BB002406E057F8240060
:101700003146FFF799FF601CC4B2AC42F6D3002407
:1017100005E03146002000F02BF8601CC4B2142C08
:10172000F7DB00201149088005EB4500C0001430AC
:1017300081B20D482838FFF771F901210A4828388D
:10174000FFF782F800BF4FF40070FFF733F900286D
:10175000F9D0002104482838FFF776F84FF40070DC
:10176000FFF764F8BDE8F08158000240B4000020A3
:10177000012905D1094A0A4B1B8822F8130006E00B
:10178000022904D1074A064B1B8822F81300044A99
:101790001288521C024B1A8070470000B2000020D1
:1017A000B4000020C00200200548817A19B105214B
:1017B000044A116002E00121024A116070470000F2
:1017C000C00A0020D001002000BFFEE7704770472C
:1017D00070B5002100230F22C47804B3154C24688F
:1017E00004F4E064C4F5E064210AC1F10403CA40D2
:1017F000447804FA03F184781440214309010E4C23
:101800000678A155047804F01F050124AC40057842
:101810006D11AD0005F1E025C5F8004109E004783F
:1018200004F01F050124AC40044D0678761145F8FC
:10183000264070BD0CED00E000E400E080E100E037
:1018400002490143024A1160704700000000FA0596
:101850000CED00E070B50226474800684478464821
:101860000068007800F07F00002844D1092C03D1E3
:1018700000F008FE06465FE0052C14D13E480068E3
:10188000C0787F280BDC3C480068807838B93A483B
:101890000068808818B938480068807A08B108253F
:1018A00065E0002648E0032C0ED133480068C0787C
:1018B000012807D130480068808818B900F006FE7A
:1018C000064639E0022637E0012C35D12A48006867
:1018D000C07801280DD128480068808848B926487A
:1018E0000068407A00F0200018B100F057FC06466E
:1018F00022E0022620E020480068007800F07F0007
:10190000012805D10B2C17D100F05CFE064613E030
:1019100019480068007800F07F0002280BD1012CE4
:1019200003D100F03BFC064606E0032C04D100F096
:10193000E1FD064600E002264EB1E0B20F4A126811
:10194000516988470646032E01D109250FE00EB1E3
:1019500008250CE0062500210948006880B2801C9B
:10196000084A42F8101030200749088000BF024999
:1019700009680D7270BD0000C0000020C400002086
:10198000505C004000600040D200002010B51148BB
:101990000068047A022C01D0042C01D1082412E042
:1019A000032C01D0052C05D1FFF79AF809480068EF
:1019B000047A08E0072C05D107490968C868804700
:1019C000082400E00824034909680C7200F01CF8A0
:1019D00010BD0000C0000020C4000020F0B5561C5F
:1019E0007510074E06EB41042B4605E034F8047BE6
:1019F00020F8017B401C5B1E002BF7D1F0BD0000DE
:101A0000006000407047000010B50D4890F82C10A1
:101A1000002000F01FFA0B480068007A082805D162
:101A200040020949088010200849088005480068DC
:101A3000007A092801D1012010BD0020FCE7000038
:101A40003C010020C0000020D0000020D200002077
:101A500010B5012001F0E9F801240B4804600020D2
:101A60000A49088008460088074908600020091DC7
:101A700008604FF4E0500549088008460088024994
:101A80000860002010BD0000405C0040CA0000203B
:101A900029B1064A52690243044B5A6104E0034AE1
:101AA00052698243014B5A617047000000100240A6
:101AB00029B1064AD2690243044BDA6104E0034AC1
:101AC000D2698243014BDA61704700000010024086
:101AD00029B1064A12690243044B1A6104E0034A21
:101AE00012698243014B1A617047000000100240E6
:101AF00029B1064A92690243044B9A6104E0034A01
:101B000092698243014B9A617047000000100240C5
:101B100029B1064AD2680243044BDA6004E0034A62
:101B2000D2688243014BDA60704700000010024027
:101B300030B500210022002400232D4D6D6805F0F2
:101B40000C0121B1042905D0082923D105E0294D34
:101B5000056022E0284D05601FE0254D6D6805F405
:101B60007012234D6D6805F48034022505EB924216
:101B70001CB9224D554305600BE01D4D6D6805F401
:101B800000351DB11E4D5543056002E01A4D554309
:101B9000056002E0174D056000BF00BF144D6D6881
:101BA00005F0F0010909174D6B5C0568DD404560E3
:101BB0000F4D6D6805F4E061090A124D6B5C4568D4
:101BC000DD4085600A4D6D6805F46051C90A0D4D10
:101BD0006B5C4568DD40C560054D6D6805F44041AE
:101BE000890B094D6B5CC568B5FBF3F5056130BD2C
:101BF0000010024000127A00001BB70000093D00EF
:101C0000808D5B0014000020240000200149086042
:101C100070470000D800424270B50546072D01D03C
:101C20002E4805702D48007808284ED2DFE800F0D5
:101C300004111A202B384E4F2948006828B900F0AB
:101C400053F806202549087002E005202349087052
:101C500041E000F049F804202049087001202049A3
:101C6000086038E002201D4948700320087032E007
:101C70001A484078401E194948700846407808B90B
:101C80000420087027E01748006884B244F010046C
:101C9000144804600520114908700A2048701AE0B1
:101CA0000E484078401E0D4948700846407858B9A3
:101CB0000C48006884B224F010040A48046006202E
:101CC000087000200649086005E000BF00BF06203C
:101CD0000249087000BF00BF70BD0000D5010020A0
:101CE000D8010020405C004010B50748006884B26D
:101CF00024F0040404480460FFF756FD4FF43F400D
:101D00000149086010BD0000405C004021B102881C
:101D100042F04002028004E002884FF6BF731A408E
:101D2000028070471AB183880B43838002E0838866
:101D30008B4383807047000010B5044611488442ED
:101D400008D101218014FFF7E3FE0021A014FFF762
:101D5000DFFE16E00C48844208D101210014FFF791
:101D6000B7FE00212014FFF7B3FE0AE007488442C3
:101D700007D10121C013FFF7ABFE0021E013FFF7ED
:101D8000A7FE10BD0030014000380040003C00407C
:101D900010B50022028802F441520B884C8823437C
:101DA0008C882343CC8823430C8923434C892343C9
:101DB0008C892343CC8923431A430280838B4FF2BF
:101DC000FF74234083830B8A038210BD7047000099
:101DD0004FF6F8710140014A11607047505C0040B5
:101DE00030B501460F4B1A78002014E003060E4C64
:101DF00004EB9353D3F8003C48F68F74234048F229
:101E000080042343C4B223430406074D05EB9454D6
:101E1000C4F8003C401C9042E8D341F08003034CDE
:101E2000236030BD38010020005000404C5C004071
:101E300010B54A105300054A126892B202EBC00274
:101E4000121D034C44F8123010BD0000505C0040DD
:101E50000060004010B502460F48006880B200EBF9
:101E6000C200801D0D4C04EB40033E290BDD4811E0
:101E700001F01F040CB9441EA0B24FF4004444EA20
:101E800080241C6007E0481001F001040CB1441CE0
:101E9000A0B284021C6010BD505C00400060004095
:101EA00030B50E4C04EB8003D3F8003C4BF68F7436
:101EB00003EA040201F480530BB182F4805201F46E
:101EC00000530BB182F4005242F4004343F080030C
:101ED000024D05EB8004C4F8003C30BD00500040CA
:101EE00010B50B4B03EB8002D2F8002C4BF68F732E
:101EF00002EA030181F4805181F4005141F400426F
:101F000042F08002024C04EB8003C3F8002C10BDA9
:101F10000050004010B54A105200044B1B689BB2A1
:101F200003EBC003024C44F8132010BD505C00408A
:101F300000600040044A126892B202EBC002921C98
:101F4000024B43F812107047505C004000600040A4
:101F500030B50E4C04EB8003D3F8003C48F6BF7458
:101F600003EA040201F010030BB182F0100201F049
:101F700020030BB182F0200242F4004343F08003BF
:101F8000024D05EB8004C4F8003C30BD0050004019
:101F900010B50B4B03EB8002D2F8002C48F6BF7350
:101FA00002EA030181F0100181F0200141F40042B6
:101FB00042F08002024C04EB8003C3F8002C10BDF9
:101FC0000050004010B5074B03EB8002D2F8002C04
:101FD00048F68F131A400A43024C04EB8003C3F8FF
:101FE000002C10BD0050004010B500F001F810BDED
:101FF0000CB50020019000903348006840F4803018
:102000003149086000BF3048006800F4003000909B
:102010000198401C0190009818B90198B0F5A06F84
:10202000F1D12948006800F4003010B1012000907F
:1020300001E0002000900098012843D12348006867
:1020400040F01000214908600846006820F00300B5
:1020500008600846006840F0020008601A484068BE
:10206000194948600846406848600846406840F49E
:10207000806048600846406820F47C10486008464C
:10208000406840F4881048600846006840F080705E
:10209000086000BF0C48006800F000700028F9D00C
:1020A0000948406820F00300074948600846406836
:1020B00040F00200486000BF0348406800F00C0098
:1020C0000828F9D10CBD0000001002400020024099
:1020D00010B50020FFF79AFD0121C805FFF7E8FCC5
:1020E00010BD000038B501242948006880B2001DE9
:1020F000284931F8100080B201EB400000902648DA
:102100000068007A092832D00098007822490968CE
:1021100008700098401C0090009800781E490968DB
:1021200048700098401C0090009800EB440000901C
:10213000009931F8020B0091FEF7E6F9164909689B
:102140004880009800EB44000090009931F8020BA1
:102150000091FEF7D9F9104909688880009800EBD2
:1021600044000090009800880B490968C88001204D
:1021700009490968087208480068C08810B9FFF763
:1021800069FB01E0FEF70AFDFFF73EFC38BD0000E9
:10219000505C004000600040C00000202DE9F04786
:1021A00054480068007800F07F08B8F1000F0AD1A9
:1021B00050480068407A00F0DF004E4909684872D4
:1021C0000020BDE8F087B8F1020F7CD149480068D3
:1021D000408818B947480068007908B10220F0E744
:1021E000DFF8149143480068477927F080052C46B2
:1021F00040480068407900F0800038B13F4901EB69
:102200008400D0F8000C00F0300606E03B4901EBFA
:102210008400D0F8000C00F4405699F80000A84261
:1022200004D91EB133480068807A08B90220C8E793
:1022300007F0800080B1314901EB8400D0F8000C38
:1022400000F0300010284BD1E0B2FEF7C1FAE0B246
:102250003021FFF77DFE43E0284901EB8400D0F8F0
:10226000000C00F44050B0F5805F39D1E4B9244A45
:1022700092F82C10E0B2FFF7EDFD204A02EB84014A
:10228000D1F8001C4BF68F7201EA020080F48050F6
:1022900080F4005040F4004141F08001174B03EB03
:1022A0008402C2F8001C1BE0E0B2FEF777FA134A82
:1022B00002EB8401D1F8001C4BF68F7201EA020098
:1022C00080F4805000E011E080F4005040F40041C0
:1022D00041F08001094B03EB8402C2F8001C00BFEF
:1022E000084909684869804700206AE700BF022062
:1022F00067E70000C00000203801002000500040C7
:102300003C010020CC00002010B504462CB901206F
:10231000064909680882002010BD05490968086857
:102320008047024800680A30F6E70000C00000203D
:10233000CC00002010B5024606480068438A32B936
:102340008888C01A034C24682082002010BD0868C9
:102350001844FBE7C000002010B504462CB901204A
:10236000064909680882002010BD05490968886887
:102370008047024800680C30F6E70000C0000020EB
:10238000CC00002010B504462CB902203949096858
:102390000882002010BD00203749088035480068B9
:1023A000007800F07F0018BB32490968487A00F0D5
:1023B000200131B13049097841F002012E4A1170F3
:1023C00005E02D49097801F0FD012B4A117000F05C
:1023D000400131B12849097841F00101264A1170C4
:1023E00005E02549097801F0FE01234A11703AE021
:1023F00020480068007800F07F00012801D11E48C5
:10240000C8E71C480068007800F07F00022828D147
:10241000184A1268517901F00F0001F080027AB178
:10242000164B03EB8002D2F8002C02F03002102A87
:1024300016D1114A127842F001020F4B1A700FE0C8
:102440000E4B03EB8002D2F8002C02F44052B2F59E
:10245000805F05D1084A127842F00102064B1A70DB
:1024600001E0002096E706490968086980470248AC
:1024700090E70000C0000020B6000020005000409F
:10248000CC00002010B50E480068C0780D4949788E
:10249000884213DC0A480068807878B908480068E8
:1024A000808858B906480068C0780549096888726C
:1024B0000549096848688047002010BD0220FCE7F4
:1024C000C000002038010020CC00002010B50748D3
:1024D0000068407A40F020000449096848720449C5
:1024E0000968C8698047002010BD0000C0000020B6
:1024F000CC0000202DE9F0412E480068467926F0F6
:1025000080073C462B480068407900F0800038B1D5
:10251000294901EB8400D0F8000C00F0300506E0FA
:10252000254901EB8400D0F8000C00F44055234805
:102530000078A04208D91F480068408820B91DB122
:102540001C480068807A10B90220BDE8F08106F0CE
:102550008000A0B1184A02EB8401D1F8001C48F6B3
:10256000BF7201EA020080F0100040F4004141F027
:102570008001114B03EB8402C2F8001C14E00E4AE8
:1025800002EB8401D1F8001C4BF68F7201EA0200C5
:1025900080F4805040F4004141F08001064B03EB91
:1025A0008402C2F8001C00BF054909688869804799
:1025B0000020CAE7C0000020005000403801002081
:1025C000CC00002010B5174B1B68D978154B1B6841
:1025D0005879154B1B689A69904704461148006862
:1025E000807AE8B13CB90F480068007918B90D4805
:1025F0000068807808B1022010BD8CB90B490968C9
:10260000C868804707480068407906490968C87269
:1026100004480068C0780349096808730020EBE7A4
:102620000220E9E7C0000020C4000020CC00002008
:1026300038B50025002000902148006884B200BF12
:1026400009E0204901EB8500D0F8000C80B21E495A
:1026500041F825006D1C082DF3D344F4806418481C
:10266000046044F00104046024F00104046000BF2D
:102670001348001D006800F480600028F8D04FF671
:10268000FF300F49091D0860002509E00E4850F889
:10269000250080B20B4A02EB8501C1F8000C6D1CCD
:1026A000082DF3D344F0080405480460006884B2A0
:1026B00044F0040402480460FEF72CFC38BD00001E
:1026C000405C004000500040DC0A002010B500F0E3
:1026D00035F910BD30B516480068164AB0FBF2F166
:1026E000B1F1807F01D301201DE021F07F40401E29
:1026F0004FF0E022506150170F22002807DA13072D
:102700001D0E0D4B00F00F04241F1D5503E0130791
:102710001C0E0A4B1C5400BF00204FF0E0229061B9
:1027200007201061002008B100BFFEE730BD0000A7
:102730000000002040420F0018ED00E000E400E03F
:1027400010B51348006840F00100114908600846C0
:102750004068104908400E494860084600680E4924
:1027600008400B4908600846006820F48020086093
:102770000846406820F4FE0048604FF41F0088605F
:10278000FFF732FC4FF000600449086010BD000004
:10279000001002400000FFF8FFFFF6FE08ED00E029
:1027A00010B50121880700F05DF840B120480068AD
:1027B000401C1F4908600121880700F044F81D48AB
:1027C000007801282DD11C480078401C1A49087057
:1027D00008460078642829D10021000700F036F867
:1027E0004FF0E020006920F001004FF0E021086187
:1027F0001921124800F0C0FB022219210F48FEF7F0
:1028000033FF4FF0E020006940F001004FF0E0217D
:1028100008610121880700F019F8002006490870B6
:1028200004E004480078022800D000BF10BD00007A
:102830002C0000203000002031000020DC010020AE
:10284000CA4302827047CA430282704721B102889C
:1028500042F00102028004E002884FF6FE731A4043
:102860000280704730B50246002000230024158AFC
:1028700005EA0103958905EA010413B10CB10120B1
:1028800000E0002030BD1AB183890B43838102E050
:1028900083898B4383817047002202881D4B9842B5
:1028A0000ED01D4B98420BD0B0F1804F08D01B4B7F
:1028B000984205D01A4B984202D01A4B984204D144
:1028C0004FF68F731A404B881A43174B984207D024
:1028D000164B984204D04FF6FF431A40CB881A4358
:1028E00002808B8883850B8803850A4B98420BD026
:1028F000094B984208D00E4B984205D00D4B984298
:1029000002D00D4B984201D10B7A038601238382BA
:1029100070470000002C01400034014000040040DA
:1029200000080040000C004000100040001400406F
:102930000040014000440140004801400448006854
:1029400020B103480068401E01490860704700003C
:102950003400002010B540F225510B4800F09BF8E0
:1029600080B1094800F052F9C4B2084801780078F3
:10297000401C064A1070064844540A2C02D101201B
:102980000449087010BD000000440040B000002061
:10299000B6020020AE00002001F40072B2F5007F04
:1029A00000D100BFCA430280704710B50022002347
:1029B00040F66A14A14200D100BF0A1201249440DB
:1029C000A3B2DC43048010BD21B1828942F40052DD
:1029D000828104E082894DF6FF731A40828170473C
:1029E00010B504462048844209D101218803FFF72D
:1029F0008FF800214FF48040FFF78AF832E01B483F
:102A0000844209D101214804FFF762F800214FF404
:102A10000030FFF75DF825E01548844209D1012117
:102A20008804FFF755F800214FF48020FFF750F895
:102A300018E01048844209D10121C804FFF748F882
:102A400000214FF40020FFF743F80BE00A488442CE
:102A500008D101210805FFF73BF800214FF4801051
:102A6000FFF736F810BD0000003801400044004078
:102A700000480040004C004000500040024600204A
:102A8000B1F5007F00D100BF13880B400BB10120CE
:102A900000E00020704770B50246002400230025A6
:102AA000002040F66A16B14200D100BFC1F34215C2
:102AB00001F01F03012606FA03F3012D02D19689C6
:102AC000334006E0022D02D1168A334001E0968A97
:102AD00033400C12012606FA04F41688344013B170
:102AE0000CB1012000E0002070BDF0B503460024C9
:102AF00000260025002040F66A17B94200D100BF29
:102B00001846C1F3421401F01F06012707FA06F523
:102B1000012C01D10C3004E0022C01D1103000E076
:102B200014301AB107682F43076002E00768AF430B
:102B30000760F0BD2DE9F04786B005460E4600243B
:102B4000A24600BFA1460027B08900B100BF2F46B2
:102B50002C8A4CF6FF700440F08804432C82AC8928
:102B60004EF6F3100440B088318908437189084358
:102B70000443AC81AC8A4FF6FF400440B089044363
:102B8000AC8201A8FEF7D4FF1F48874202D1DDF8CE
:102B900010A001E0DDF80CA0A88900F4004040B1CD
:102BA0000AEBCA0000EB0A1031684900B0FBF1F8EB
:102BB00007E00AEBCA0000EB0A1031688900B0FB9D
:102BC000F1F86420B8FBF0F004012009642101FB56
:102BD0001089A88900F4004040B1322000EBC90000
:102BE000B0FBF1F000F00700044308E0322000EBF6
:102BF00009106421B0FBF1F000F00F0004432C81B8
:102C000006B0BDE8F0870000003801400146888822
:102C1000C0F308007047C1F308028280704710B506
:102C20004FF48020FEF726F910BD704710B5084814
:102C300008490860022009680872074807490860C7
:102C4000074808490860054909680868804710BDB9
:102C5000C00A0020C00000203C010020C400002069
:102C60006C010020CC0000200EB54FF48020FEF750
:102C700001F94FF48020009008208DF80500012014
:102C80008DF806006846FEF7FBF814208DF8080062
:102C900001208DF8090000208DF80A0001208DF830
:102CA0000B0002A8FEF794FD2A208DF808000020F2
:102CB0008DF8090002A8FEF78BFD0EBD10B588B097
:102CC000002468480068684908800846008800F4C5
:102CD000004066490988084008B1FDF71BFC6248BE
:102CE000008800F4806061490988084030B14FF6DF
:102CF000FF305C4908605E49486880475A48008850
:102D000000F4005059490988084018B14DF6FF7089
:102D1000544908605448008800F480505349098899
:102D2000084030B14EF6FF704E4908600020FEF7B3
:102D300073FF4D48008800F400604C490988084042
:102D400060B14C48007810B1FFF772FC02E002203D
:102D5000FEF762FF4FF2FF70424908604248008868
:102D600000F4007041490988084040B14FF6FF5017
:102D70003C49086040480078401C3F4908703A4888
:102D8000008800F48070394909880840002866D01E
:102D90004FF6FF6033490860081D006800F40040EA
:102DA000002856D035480068401C34490860084661
:102DB0000068032850D92B48001F006800F0080065
:102DC000002849D12748001F006880B22C490860BC
:102DD000002408E02B4901EB8400D0F8000C80B2FD
:102DE0004DF82400641C082CF4D32548006840F0FA
:102DF0000100234908600846006880B21949091F8C
:102E000008601F48006820F001001D49086008465E
:102E1000006880B21349091F086000BF11480068AC
:102E200000F480600028F9D04FF6FF300D490860AB
:102E3000002408E05DF8240080B2124A02EB84010D
:102E4000C1F8000C641C082CF4D300200B49086066
:102E500002E00020094908600720FEF7DDFE08B007
:102E600010BD0000445C0040F0000020CA000020BB
:102E70003C010020D4010020F2000020F4000020DA
:102E8000F80000200050004010B5FFF717FF10BDFC
:102E900038B5044601210420FEF72AFE74B14FF430
:102EA000C050ADF8000003208DF8020018208DF806
:102EB000030069460B48FEF774F812E04FF4C05067
:102EC000ADF8000003208DF8020010208DF80300FB
:102ED00069460448FEF765F84FF4C0510148FEF713
:102EE0003CF938BD000801400020064908604FF455
:102EF0003F4005490880084600880249091F0860CC
:102F000000207047445C0040CA0000202DE9F041D9
:102F100004460E46154604F07F00FEF733F90746D7
:102F2000AAB23946304600F00BF8A9B204F07F008F
:102F3000FFF700F80020BDE8F08100BFFEE70000C9
:102F4000F0B5144604F1010C4FEA6C07DFF824C019
:102F50000CEB41033D460AE00678401C90F800C0A7
:102F600046EA0C2223F8022B9B1C401C6D1E002DF0
:102F7000F2D1F0BD0060004010B50A4603680021A0
:102F800005E04C1C50F8244040F82140491C914277
:102F9000F7D3541E40F8243010BD00000025532400
:102FA00000BF0AE02A4840F825406400B4F5000F4D
:102FB00001D96FF05304681CC5B2192DF2DBFFF77D
:102FC000BFFB01210920FEF793FD01212148FEF7F7
:102FD00073F8FFF77FFBFEF791FA19211C48FFF702
:102FE000CBFF022219211A48FEF73EFBFDF798FF9E
:102FF00000F0E0F800F0E6FBFDF7C2F9FDF772FA29
:103000000C211548FDF74AFA21E01448007888B1F0
:1030100000F0ACF912480078012818D100201049BE
:10302000087010480068052811D10B48001DFEF7F4
:1030300059FA0CE000F09AF909480078012806D105
:103040000020074908700C210348FDF727FADCE748
:10305000DC01002000023000A20000202800002037
:103060009F000020D001002070B504460D4604EBFF
:103070008401404A02EB810151F825003EA1FDF791
:10308000EBF830B93E48007840F002003C49087047
:103090006EE004EB8401374A02EB810151F8250010
:1030A00038A1FDF7D9F830B93548007840F0200054
:1030B000334908705CE004EB84012E4A02EB810185
:1030C00051F8250031A1FDF7C7F830B92C48007838
:1030D00040F001002A4908704AE004EB8401254AC7
:1030E00002EB810151F825002AA1FDF7B5F830B9AE
:1030F0002348007840F010002149087038E004EBC4
:1031000084011C4A02EB810151F8250023A1FDF73F
:10311000A3F830B91A48007840F004001849087044
:1031200026E004EB8401134A02EB810151F82500EB
:103130001CA1FDF791F830B91148007840F040002B
:103140000F49087014E004EB84010A4A02EB810184
:1031500051F8250015A1FDF77FF830B9084800782F
:1031600040F008000649087002E00020104908708D
:1031700070BD0000380000204C5368696674000080
:103180009C00002052536869667400004C437472BE
:103190006C000000524374726C0000004C416C746F
:1031A0000000000052416C740000000057696E007E
:1031B0009E00002008B501210C20FEF799FCF820A4
:1031C000ADF8000003208DF8020028208DF80300E0
:1031D00069460848FDF7E5FE7320ADF800000320BE
:1031E0008DF8020010208DF8030069460248FDF7B3
:1031F000D8FE08BD000C01400008014010B50020B9
:103200001CE0002111E000EB8002194B1A445256D9
:1032100000EB8003174C23445B569A4203D00122F3
:10322000154B1A7003E04A1CD1B20529EBDB00BF35
:10323000114A127802B103E0421CD0B20528E0DB4B
:1032400000BF002011E000210BE000EB8002094BE1
:103250001A44525C00EB8003054C23445A544A1C28
:10326000D1B20529F1DB421CD0B20528EBDB10BD41
:103270006B020020520200209D00002010B50024A7
:1032800006E0054A2146054800F00AF8601CC4B271
:10329000052CF6DB10BD0000BE3800080008014018
:1032A00070B506460C46154635F814103046FDF745
:1032B00056FF3220FDF7CCFD08212A48FDF744FFD8
:1032C00018B1FF202849085502E00020264908557A
:1032D0003220FDF7BDFD10212248FDF735FF20B15A
:1032E000FF212148401D015503E000211E48401DDB
:1032F00001550120FDF7ACFD20211A48FDF724FF00
:1033000020B1FF2118480A30015503E0002116487A
:103310000A3001550120FDF79BFD40211148FDF7C2
:1033200013FF20B1FF2110480F30015503E00021A9
:103330000D480F3001550120FDF78AFD8021094815
:10334000FDF702FF20B1FF2107481430015503E0CB
:10335000002105481430015535F814103046FDF7AA
:10336000FCFE70BD000C01405202002010B5FFF7BA
:1033700085FFFFF743FF0648007838B10020044975
:10338000087000F009F801200249087010BD000023
:103390009D0000209F0000202DE9F0419AB04FF0E1
:1033A00000080020F6490870F64890F90000401C1B
:1033B00000287DD10024F34890F91300401C002818
:1033C00039D1F148007808B9012000E00020EE4929
:1033D000087000214FF08040FFF738FAEA48007883
:1033E00038B9FDF77FF802221921E848FEF73CF9C9
:1033F00006E0FCF7CDFF02221921E548FEF734F97B
:1034000040F2DC50FDF717FD01218807FFF71EFA97
:10341000E0480078022809D1642101A8FCF7F4FEF5
:103420000222192101A8FEF71FF91DE1D9480078F1
:103430000328FAD158E0D34890F90400401C002832
:103440003ED1642101A8FCF7DFFED24800780328B2
:103450000BD10222192101A8FEF706F90220CD495D
:1034600008700120CC49087029E0CB48007840B9A9
:103470000222192101A8FEF7F7F80220C5490870B9
:1034800013E0532000240AE0C44941F8240040001E
:10349000B0F5000F01D96FF05300611CCCB2192CAC
:1034A000F2DB0121BB4A117000BFBB48007800E08D
:1034B000DDE008B9012000E00020B7490870D3E042
:1034C000B04890F91400401C00287BD10320B1497A
:1034D0000870B3480078401CC0B2B1490870082891
:1034E00001D10020087000BFAD480078082814D230
:1034F000DFE800F0041425364758697A002405E017
:10350000FF20A64941F82400601CC4B2192CF7DB47
:1035100002221921A148FEF7A7F875E0002406E071
:103520004FF47F409D4941F82400601CC4B2192C1F
:10353000F6DB022219219948FEF796F864E0002490
:1035400006E04FF47F00954941F82400601CC4B2A6
:10355000192CF6DB022219219048FEF785F853E07A
:10356000002406E04FF6FF708C4941F82400601CEF
:10357000C4B2192CF6DB022219218848FEF774F830
:1035800042E0002406E04FF0FF10844941F8240097
:10359000601CC4B2192CF6DB022219217F48FEF709
:1035A00063F831E0002405E07E487C4941F82400BE
:1035B000601CC4B2192CF7DB022219217748FEF7F0
:1035C00053F821E021E0002406E06FF07F407349CA
:1035D00041F82400601CC4B2192CF6DB0222192128
:1035E0006E48FEF741F80FE0002405E06E486B4995
:1035F00041F82400601CC4B2192CF7DB0222192107
:103600006648FEF731F800BF2EE05E4890F91600DC
:10361000401C90B95F480078012825D1002409E0BA
:103620005E4850F82400614908445C4941F8240090
:10363000601CC4B2192CF3DB16E0524890F9170055
:10364000401C88B95348007801280DD1002409E0B6
:10365000524850F824005649401A504941F8240075
:10366000601CC4B2192CF3DB1AB0BDE8F081002550
:1036700019E005EB45004F49085C90B105EB4500AA
:103680000844407800EB80003E49084405EB4501C2
:10369000484A11448978405C18B9002005EB45017F
:1036A0005054681CC5B2062DE3DB002552E000270C
:1036B0004CE005EB850033490844C057401CC0BBB3
:1036C00039462846FFF7D0FC3B48007888BB0026E7
:1036D0000FE006EB46003749085C05EB8501374AE9
:1036E0001144C95D884202D14FF0010803E0701C0B
:1036F000C6B2052EEDDB00BFB8F1000F1FD10026CA
:103700001AE006EB46002B49085C98B905EB8500EA
:103710002A490844C05D06EB4601264A505406EB90
:10372000460011460844457006EB46000844877081
:1037300004E009E0701CC6B2062EE2DB01E04FF0A7
:10374000000801201C490870781CC7B2052FB0DBA7
:10375000681CC5B2052DAADB094800781849087114
:10376000002608E006EB46001249095CB01D144A29
:103770001154701CC6B2062EF4DB00BF74E70000C3
:103780009C00002052020020280000204038000841
:10379000DC37000830000020A0000020DC01002001
:1037A000A100002000FFFF00BB5599000F0F0F0084
:1037B000F0F0F000400200209E000020A438000835
:1037C000A200002010B50120FFF762FBFFF74CFAC2
:1037D000FEF77EFCFFF72AFA10BD00000000000093
:1037E00000000000000000000000000000000000D9
:1037F00000000000FFFFFF0000000000FFFFFF00CF
:103800000000000000000000FFFFFF0000000000BB
:10381000FFFFFF000000000000000000FFFFFF00AE
:10382000FFFFFF00FFFFFF0000000000000000009E
:103830000000000000000000000000000000000088
:1038400000000000FF000000FF000000FF0000007B
:103850000000000000000000FF0000000000000069
:10386000FF0000000000000000000000FF0000005A
:10387000FF00000000000000000000000000000049
:10388000FF00000000000000FF000000000000003A
:1038900000000000FF000000FF000000FF0000002B
:1038A00000000000294A4D4B4E2A5F5C596254606B
:1038B0005D5A6255615E5B63565757585800010068
:1038C0000200100020004000120100020000004031
:1038D00078671201000201020301090229000101B7
:1038E00000C0320904000002030101000921100197
:1038F0002101223D000705810308000A0705010395
:1039000001000A05010906A101050719E029E715CB
:1039100000250195087501810295017508810395BF
:1039200006750825FF190029658100250195027596
:10393000010508190129029102950175069103C03C
:10394000040309042603430061006C006C0020009E
:103950004D006500200046006100740068006500AD
:103960007200000000000000000028034200D97A25
:103970003A006753D2522A4E0856200020007600A3
:1039800031002E003100005F906E0000000000004A
:10399000000000002A0000002B0000002D000000A5
:1039A0002E0000002F000000300000003100000059
:1039B0003200000033000000340000003500000039
:1039C0003600000037000000380000003900000019
:1039D000454E4400484F4D450000000045736300CC
:1039E0004261636B737061636500000050616765DD
:1039F000446F776E000000005061676555700000ED
:103A0000456E746572000000283A0008000000202E
:103A1000DC01000028010008083B0008DC01002050
:103A2000840F0000840100081184A24A046809017F
:103A3000020304060708090C69106E020406080157
:103A4000247113DC391B08D4041AD0041AF8041AA0
:103A5000EC041AE0041AC4041AB8041AAC041AA834
:103A6000041AA4041AC8041ABC045AB0141A940400
:103A70001ACC041AC0041AB4041AA0041A9C045ADA
:103A80009804115A3A04396E120C6AA1750127156F
:103A9000011A03531254124D1233021C3213690ED1
:103AA0000C3008CF1704411A029413BD141408D91E
:103AB000131B08B9081ABB04138D121B08B5101A82
:103AC0009D041A1D041A09041A7504413240293C48
:103AD0001A7D280916581A951C13C8383308121A6B
:103AE000DA08322913033933083D1AEC102A094841
:103AF000191032041A440832261A6A08322822D5CC
:083B000073201A199B5100000B
:04000005080000ED02
:00000001FF
